:1000000025000A0C0600000C02000604A6044604A3
:1000100086046606130A26060E0A100AA60486043B
:10002000A6058605090A3E092606240A3809260778
:10003000240A3E092606240A38092607240A3E090E
:100040002606240AA605250AA6045A092606360A03
:1000500038092607360A5A092606360A38092607B5
:10006000360A5A092606360A8605090A8604090A46
:10007000C30C29000000E9023A0A0008180C290004
:100080000605000000000000000000000000000065
:100090000000000000000000060400000000000056
:1000A0000000000000000000000000000000E90265
:1000B000400A0008180C2900460500000000000056
:1000C0000000000000000000000000000000000030
:1000D00046040000000000000000000000000000D6
:0C00E000000000000000E9025C0A0008BB
:021FFE00EA0FE8
:00000001FF
